:04000000B601CD294F
:100008000800B616B61EB612B6190E28B615472041
:10001800031835280830A3005B20A20DA30B102875
:10002800B61E402065206120B61A35203A202208E5
:100038000310C829B616B61EB61236192828FE3976
:10004800B70036150310C829361A3028A600361608
:1000580047200318352826084E2003183528B61ED1
:10006800C8294020652036113612B6113A08840096
:1000780038088417800446283A088400380980051F
:100088008417800508003A20652040206120370841
:10009800B6190138A2000830A300A20D03183A20AF
:1000A800031C402065206120A30B51283A206520BD
:1000B8003A08840038080005FF3E3B0884003909E7
:1000C80043283B08840039083D2864007F20031832
:1000D8006928CE20A8010830A300CF207F2003186C
:1000E800A80AAB1EA801A20CA30B7128AB1AA21375
:1000F800CF20220808003A088400380884178004B2
:10010800841300052B1B3806FF3E0800A4002908AD
:100118000319C829C321A0002518831724088400BF
:10012800200880008313A40AA9038B280408A600CA
:100138003A0884008030B7050830A7000310031878
:10014800B70AB420A60CA70BA3280000AB1A370CDB
:10015800B420CB210314B4202F08A3002E082F2984
:100168008413AB1FC328000838042B1F38068000EF
:10017800841700083804031C38068000CF280008BC
:100188003804031C38062B1B3806800084173809EE
:100198008005CF2837172B081F39003EA1002A08F1
:1001A8000E3E0318A10A371F3C293713A00002305E
:1001B80060213C29B71329080319B7170430A80090
:1001C800250EEB202508EB20240EEB2024080F3900
:1001D800F63E0318073E0A3EF128A000A8030319BB
:1001E800B71329080319FB28280203180800200858
:1001F800031DB713B71B0800303EC32983178001BE
:10020800840AFF3E031D0329C82921082004031975
:10021800A00A8030201AA1062019A106A018A1065C
:10022800210DA00DA10DC82903178D0083168C136D
:100238000C1483120C08C82903178C0083168C131E
:100248000C1555308D00AA308D008C148C182A2975
:100258000C11C829A301A200FF30A207031CA307A1
:10026800031CC8290330A100E6303C213029A10134
:10027800FC3EA000A109031C4729FF300000A0078D
:1002880003184229A0076400A10F41290800013E74
:10029800A7000A30A200A3019121A70B5029240826
:1002A80008000310A00DA10DFF3E031855292008D2
:1002B800C8290310A10CA00CFF3E03185D292008D3
:1002C800C829A101A301A20002307A29A301A20032
:1002D80003307A29A301A20001307A29A301A200E0
:1002E80006307A29A101A301A2000530A80023083D
:1002F8002102031D8129220820020430031801303D
:10030800031902302805031DFF30C8290038031DD2
:10031800FF300405031DFF30C829A501A4011030D2
:10032800A600210DA40DA50D2208A4022308031C74
:10033800230FA5020318A7292208A40723080318D6
:10034800230FA5070310A00DA10DA60B95292008C2
:10035800C8291030A800A101A001A70CA60C031CF5
:10036800BB292208A00723080318230FA107A10C03
:10037800A00CA50CA40CA80BB1292408C82984003A
:1003880031088A0030088200831303138312640043
:1003980008002030840060308A010321A0308400E6
:1003A80050308A0103211030840060308A01022114
:1003B8009030840060308A010221831607309F0044
:1003C800990183129801831602309800EE01EF011B
:1003D800E301E20106108610061188018710071054
:1003E8000711871205128512DB01CE01C301013006
:1003F800CD00E801C430E700C201CE01C301E80125
:10040800C430E7008312880107148714071587167C
:10041800891009150130A300F4308A012F218316B1
:10042800DB01B0011030B100B401B50164005B0814
:10043800003C8A110A128312031D312A83160830E0
:10044800BA000730B9002030AE00AF012030B2004A
:10045800B30183128A110A123D2A83160630BA00A4
:100468000530B9002830AE00AF012830B200B30122
:100478008312091164308A012E2109158A150A127E
:10048800312B8A110A126C2283165C0883128800A9
:100498008712871407110710071407158A110A1203
:1004A8006C2283165D08831288008712871407114F
:1004B8000710071407158A110A126C2283165A08A6
:1004C80083128800871407110710071407150800FE
:1004D80007158316FF308800831287160714071143
:1004E8008710003008180130A00001308A017621F9
:1004F800B200003088180130A00001308A0176214E
:10050800B4003208840034088A018A218A110A1248
:10051800031D6C2A871407158316880183120800A7
:100528008A016C228316FF30880083128712871095
:10053800071102308A013B2108088316C000831284
:100548000715871483168801831208008A110A1276
:1005580050238A019422080083160130E800831290
:1005680083162A088312A60083162B088312A70075
:100578002030A200A3018A01AD21B2002508B300F2
:10058800831630088312B207831631080318013E18
:100598008312B307831628088312A000831629083C
:1005A8008312A10083163A088312A200A3018A01CC
:1005B8009121B4002108B500320834078316A00041
:1005C800831233080318013E35078316A10020085B
:1005D800A6002108A7002808CB002A08CC0021087B
:1005E800DD002008DC002430DA0083128A0145226D
:1005F800640083166808003C8A110A128312031DDE
:10060800292B831628088312A00083162908831231
:10061800A10083163A088312A200A3018A0191213E
:100628002408B2002508B300320883163902831261
:10063800B20033090318013EB300F83032048316C0
:10064800DA0083128A110A124A2B831628088312A9
:10065800A000831629088312A10083163A08831282
:10066800A200A3018A0191212408B2002508B30041
:100678003208831639028312B20033090318013E87
:10068800B300F03032048316DA0083128A015F2245
:100698008316E8018312080083162A088312A6002D
:1006A80083162B088312A7002030A200A3018A0119
:1006B800AD21B2002508B300831630088312B207B3
:1006C800831631080318013E8312B30783162808DE
:1006D8008312A000831629088312A10083163A0802
:1006E8008312A200A3018A019121B4002108B50058
:1006F800320834078316A000831233080318013E1A
:1007080035078316A1002008A6002108A7002108A4
:10071800DD002008DC002430DA0083128A0145223B
:100728000800831658085507A800A901A90D5908FB
:100738005607AA00AB01AB0D83128A01B4228316B7
:1007480058085502A800A901031CA903590856070F
:10075800AA00AB01AB0D83128A01B4228316550897
:100768005807A800A901A90D59085602AA00AB010B
:10077800031CAB0383128A01B4228316580855025E
:10078800A800A901031CA90359085602AA00AB0135
:10079800031CAB0383128A01B42283165908550738
:1007A800A800A901A90D58085607AA00AB01AB0D6E
:1007B80083128A01B422831659085502A800A90198
:1007C800031CA90356085807AA00AB01AB0D8312F6
:1007D8008A01B422831655085907A800A901A90D52
:1007E80058085602AA00AB01031CAB0383128A0106
:1007F800B422831659085502A800A901031CA903AD
:1008080058085602AA00AB01031CAB0383128A01E5
:10081800B422080083163108DD003008DC004230BD
:10082800DA0083128A01452283162F08DD002E087C
:10083800DC004330DA0083128A014522831635082A
:10084800DD003408DC004030DA0083128A014522DA
:1008580083163308DD003208DC004130DA008312E9
:100868008A01452283168030DA0083128A015F22CA
:100878008316DD01DC012430DA0083128A01452267
:1008880083169830DA0083128A015F2283160130BA
:10089800C30083126400F130831643028A110A12DE
:1008A80083120318792C83160130C6008312640062
:1008B8004130831646028A110A1283120318722CD9
:1008C8008316DD01C030DA0083128A0152228316B2
:1008D800C60A8A110A128312031D5B2C8316C30AE7
:1008E8008A110A128312031D4E2C83169C30DA00DB
:1008F80083128A015F2208008316D8015708D9009D
:1009080083120230A600A701831657088312A2009B
:10091800A3018A01AD21B2002508B3003208023CC8
:100928008316AC0083123308031C013E003C831677
:10093800AD00831264008316580859028A110A12FE
:100948008312031CF92C8A01952364008A110A1268
:1009580083168310AD1F831483128318D12C04309F
:10096800A600A701831658088312A200A3018A01D2
:10097800AD21B2002508B3000630B2070318B30A48
:1009880032088316AC07831233080318013E831616
:10099800AD0783128A110A12F42C831659085802DB
:1009A8008312B200B301031CB3030430A600A701ED
:1009B8003208A2003308A3008A01AD21B20025083D
:1009C800B3000A30B2070318B30A32088316AC071B
:1009D800831233080318013E8316AD07D903831227
:1009E8008316D80A83128A019E2C08008316D80120
:1009F8005708D90083120230A600A70183165708AA
:100A08008312A200A3018A01AD21B2002508B30018
:100A18003208023C8316AC0083123308031C013EE3
:100A2800003C8316AD0083126400831658085902EF
:100A38008A110A128312031C4A2D8A0195238316F0
:100A4800590858028312B200B301031CB3030430DF
:100A5800A600A7013208A2003308A3008A01AD212D
:100A6800B2002508B3000A30B2070318B30A3208E7
:100A78008316AC07831233080318013E8316AD07AB
:100A88000330D902D80A83128A01182D08008A1166
:100A98000A12592683164F085002C80052085302FA
:100AA800C9006400490848028A110A128312031C0B
:100AB800DB2D831649088312A000A10102308A01A8
:100AC8005821B2002108B300831648088312320265
:100AD8008316AC0083123308031CFF3E8316AD0057
:100AE8005208AA00AB0149088312A000A1010230F4
:100AF8008A0158218316A200831221088316A300B5
:100B0800480849028312B200B301031CB303023040
:100B1800A600A7013208A2003308A3008A01AD216C
:100B28008316A400831225088316A5004F08A80081
:100B3800A9018312831628088312A00083162908A6
:100B48008312A1008316500883128A016E218A112C
:100B58000A12031DDA2D64008A110A128316831003
:100B6800AD1F831483128318C42D83162208AC0783
:100B780023080318013EAD0783128A110A12CF2DEC
:100B880083162408AC0725080318013EAD07AA0AF6
:100B98000319AB0A83128A01B4228316A80A03191F
:100BA800A90A8A110A128312031D9E2D08008316B2
:100BB80048088312A000A10102308A015821B2001E
:100BC8002108B30083164908831232028316AC0049
:100BD80083123308031CFF3E8316AD004F08A8009C
:100BE800A90148088312A000A10102308A015821F6
:100BF8008316A200831221088316A300490848021D
:100C08008312B200B301031CB3030230A600A7018C
:100C18003208A2003308A3008A01AD218316A4007C
:100C2800831225088316A5005208AA00AB01831277
:100C380083162A088312A00083162B088312A100AA
:100C48008316530883128A016E218A110A12031D22
:100C5800582E64008A110A1283168310AD1F83145C
:100C680083128318422E83162208AC072308031820
:100C7800013EAD0783128A110A124D2E83162408ED
:100C8800AC0725080318013EAD07A80A0319A90AED
:100C980083128A01B4228316AA0A0319AB0A8A119D
:100CA8000A128312031D1C2E0800640083164F08C5
:100CB80050028A110A1283120318682E83164F08ED
:100CC8005002CF07D00283126400831652085302E1
:100CD8008A110A1283120318772E831652085302B8
:100CE800D207D3028312080083162A088312A000B1
:100CF80083162B088312A1000830A200A3018A01E1
:100D08009121B2002108B3003208A6003308A700D9
:100D18002030A200A3018A01AD21B2002508B3004A
:100D2800831634088312B207831635080318013E68
:100D38008312B307831628088312A0008316290894
:100D48008312A10083163A088312A200A3018A0124
:100D58009121B4002108B500320834078316A00099
:100D6800831233080318013E35078316A1002108B2
:100D7800DD002008DC002430DA0083128A014522D5
:100D880008008A110A12D3278A0145228A110A12F9
:100D98008027203083163B02BF0083128A01782601
:100DA80083163F08DD006708DA0083128A015222A1
:100DB8008A110A128A2708007D08A0007E08A1006F
:100DC80004308A014B218316BB0083128A110A1250
:100DD8003A2708308316A8070318A90A83127D0842
:100DE800A0007E08A10003308A014B218316BB00B6
:100DF80083128A110A123A2708308316A8070318A3
:100E0800A90A83127D08A0007E08A10002308A0189
:100E18004B218316BB0083128A110A123A27083025
:100E28008316A8070318A90A83127D08A0007E0864
:100E3800A10001308A014B218316BB0083128A115D
:100E48000A123A2708308316A8070318A90A83123A
:100E58007D08A0007E08A10000308A014B2183167E
:100E6800BB0083128A110A123A27080083163B082E
:100E7800093C8A110A128312031C5B2F8A110A1279
:100E88004B278316CE0083128A110A125B2F073074
:100E98008A0083163B088312820730343134323497
:100EA8003334343435343634373438343934203004
:100EB80083164E02BF0083128A01D22608008A11C7
:100EC8000A12D3278A110A1280278A01502383160F
:100ED8003E08DD006708DA0083128A0152228A116F
:100EE8000A128A2708008A01452283169830DA00F8
:100EF80083128A015F2208008A110A12D3278316F7
:100F08009430DA0083128A015F2208008A110A12DB
:100F1800D32783169C30DA0083128A015F220800E7
:100F2800831643085C3E840000088312B200FF3039
:100F3800A200A20A22080F3C8A110A12031CC72F1A
:100F48008A110A12B32732028A110A12031D9D2F31
:100F580022088316DE0083128A110A12C72F07306F
:100F68008A0022088207303431343234333434343E
:100F78003534363437343834393461346234633490
:100F8800643465346634080083163108DD0030089F
:100F9800DC004230DA0083128A01452208008316F9
:100FA8003508DD003408DC004030DA0083128A019D
:100FB8004522080083166B08A800A9016D08AA003D
:100FC800AB01831283162A088312A00083162B080C
:100FD8008312A10083166C0883128A016E218A1578
:100FE8000A12031D02288A01B4228316AA0A0319C9
:100FF800AB0A8A110A128312031DE62F01308316E9
:101008006B07A800A901A90D6D08AA00AB018312FE
:1010180083162A088312A00083162B088312A100C6
:1010280083166C0883128A016E218A150A12031D21
:101038002E288A01B42283166908AA078A150A127B
:101048008312031C0C288316AA0A8A150A12831213
:10105800031D0C28080083166C08AA00AB016B0856
:10106800A800A9018312831628088312A0008316FA
:1010780029088312A10083166A0883128A016E2147
:101088008A150A12031D53288A01B4228316A80A56
:101098000319A90A8A150A128312031D3728FF307B
:1010A80083166C07AA00FF300318013EAB006B08DB
:1010B800A800A9018312831628088312A0008316AA
:1010C80029088312A10083166A0883128A016E21F7
:1010D8008A150A12031D81288A01B4228316690819
:1010E800A8078A150A128312031C5F288316A80A08
:1010F8008A150A128312031D5F2808008A015926DF
:1011080083164F08C30083126400831643085002F5
:101118008A150A128312031CB82883165208C600BF
:10112800831264008316460853028A150A12831232
:10113800031CB02883164308A800A9014608AA0082
:10114800AB0183128A01B42283166908C6078A157F
:101158000A128312031C952883166908C3078A1587
:101168000A128312031C882808008A01592683164C
:101178004F08C300831264008316430850028A157F
:101188000A128312031CE12883164308A800A90148
:101198005208AA00AB0183128A01B42283165308AD
:1011A800AA00AB0183128A01B42283166908C30717
:1011B8008A150A128312031CBF2883165208C3001B
:1011C800831264008316430853028A150A12831295
:1011D800031C072983164308AA00AB014F08A8007F
:1011E800A90183128A01B42283165008A800A90114
:1011F80083128A01B42283166908C3078A150A1262
:101208008312031CE52808008316D8015708D90063
:1012180083120230A600A701831657088312A20082
:10122800A3018A01AD21B2002508B3003208023CAF
:101238008316AC0083123308031C013E003C83165E
:10124800AD00831264008316580859028A150A12E1
:101258008312031C58298A019523831659085802BA
:101268008312B200B301031CB3030430A600A70124
:101278003208A2003308A3008A01AD21B200250874
:10128800B3000A30B2070318B30A32088316AC0752
:10129800831233080318013E8316AD07D903D80A11
:1012A80083128A150A12262908008316D8015708BE
:1012B800D90083120230A600A701831657088312AB
:1012C800A200A3018A01AD21B2002508B3003208AB
:1012D800023C8316AC0083123308031C013E003C19
:1012E8008316AD00831264008316580859028A15C4
:1012F8000A128312031CA1298A0195230430A6002F
:10130800A701831658088312A200A3018A01AD2100
:10131800B2002508B3000630B2070318B30A320832
:101328008316AC07831233080318013E8316AD07F2
:10133800D80A83128A150A12772908000730BA00DA
:101348004030B8002030AA00AB01AE01AF01023036
:10135800A900831640088312A400A5019A30B000A2
:10136800B1018A01DE2008000730BA008030B800D9
:101378002030AA00AB018A0169205D3C8A150A1257
:10138800031DBF290230A9006930B000B101A501D1
:101398005C308A018A208316C301831264000230FC
:1013A800831643028A150A1283120318E9298A014F
:1013B8009427831643085C3E84005E088000C30AB5
:1013C8008A150A128312031DD2295C08A000A10104
:1013D80004308A015821B2002108B3005D083204A4
:1013E800FF0008000730BA008030B8002030AA009B
:1013F800AB018A0169205D3C8A150A12031DFD298B
:101408000430A9006930B000B101A5015C308A013F
:101418008A208316C30183126400043083164302B2
:101428008A150A1283120318272A8A019427831619
:1014380043085C3E84005E088000C30A8A150A12CD
:101448008312031D102A5C08A000A10104308A0140
:101458005821B2002108B3005D083204FF005E087D
:10146800A000A10104308A015821B2002108B3006C
:101478005F0832048316B600831208000730BA00EA
:101488008030B8002030AA00AB018A0169205D3C99
:101498008A150A12031D492A0630A9006930B000CE
:1014A800B101A5015C308A018A208316C301831229
:1014B80064000630831643028A150A128312031841
:1014C800732A8A019427831643085C3E84005E08C9
:1014D8008000C30A8A150A128312031D5C2A5C085D
:1014E800A000A10104308A015821B2002108B300EC
:1014F8005D083204FF005E08A000A10104308A01E3
:101508005821B2002108B3005F0832048316B600E0
:1015180083126008A000A10104308A015821B2009A
:101528002108B300610832048316B700831208004B
:101538000730BA008030B8002030AA00AB018A0119
:1015480069205D3C8A150A12031DA32A8A016920B5
:101558008316DE0030305E02E9005E08C0008312A8
:1015680008000730BA008030B8002030AA00AB016C
:101578008A0169205D3C8A150A12031DBC2A0830BD
:10158800A9006930B000B101A5015C308A018A2048
:101598008316C301831264000830831643028A1538
:1015A8000A1283120318E62A8A019427831643082D
:1015B8005C3E84005E088000C30A8A150A12831202
:1015C800031DCF2A5C08A000A10104308A0158211C
:1015D800B2002108B3005D0832048316CF008312DD
:1015E8005E08A000A10104308A015821B200210838
:1015F800B3005F0832048316D00083126008A0008D
:10160800A10104308A015821B2002108B300610801
:1016180032048316D20083126208A000A1010430AC
:101628008A015821B2002108B300630832048316E6
:10163800D300831208007F088316D5003608D60029
:101648003708D700831208007F088316A800A9016D
:101658003608AA00AB01831208008A010E248A0109
:101668007727F901FA018316AA01AB0183128316C1
:101678002A088312A00083162B088312A100A30155
:101688003F308A016F218A150A12031D922B831697
:10169800A801A9018312831628088312A0008316C3
:1016A80029088312A100A301EF308A016F218A154E
:1016B8000A12031D892B0730BA001030B800073012
:1016C800BB000830B900A0308A0120207A088A01BE
:1016D800202079088A0120208A0105208316BE006F
:1016E80083128A016327F90A0319FA0A0830831654
:1016F800A8078A150A128312031C4F2B8316A90AFE
:101708008A150A128312031D4F2B8316AA0A03197E
:10171800AB0A8A150A128312031D3B2B07150730E3
:10172800A300D0308A012F218A013C248A018A270C
:1017380083167730D5001F30D6000A30D7008312C1
:1017480064001F30831657028A150A128312031881
:10175800B72B8A0180240A308316D7078A150A1204
:101768008312031CA42B83162D30D5001F30D600FE
:101778000A30D700831264001F30831657028A1577
:101788000A1283120318D32B8A150A1259210A3018
:101798008316D7078A150A128312031CBF2B8316D8
:1017A800C230D5001F30D6000A30D700831264003B
:1017B8001F30831657028A150A1283120318EF2B5B
:1017C8008A150A1208210A308316D7078A150A12C1
:1017D8008312031CDB2B0730A300D0308A012F2192
:1017E8008A013C248A018A2783160830A800A901A7
:1017F8000830AA00AB01C301831264001B308316B2
:1018080043028A150A1283120318492C83164308C7
:101818001A3C8A150A128312031C3C2C8A150A12D8
:101828001B248316BB0083128A150A123C2C0C3029
:101838008A008316430883128207533461346E3456
:1018480079346F34203432343434303478343634A4
:10185800343420347534733469346E346734203446
:1018680061342034543436343934363433344334E0
:101878008A01C52608308316A8070318A90AC30ACF
:101888008A150A128312031D012C0730A300D030D9
:101898008A012F2183162830A800A9011830AA0030
:1018A800AB01C301831264001330831643028A1507
:1018B8000A1283120318972C83164308123C8A15C0
:1018C8000A128312031C8A2C8A150A1271248316A1
:1018D800BB0083128A150A128A2C0C308A008316E0
:1018E8004308831282072034423479342034433445
:1018F8004F344D345034533479347334283463348A
:101908002934203432343034303432348A01C52614
:1019180008308316A8070318A90AC30A8A150A12E9
:101928008312031D572C83162230AA00AB013030D6
:10193800A800A9018312831628088312A000831621
:1019480029088312A100A301C8308A016F218A15D2
:101958000A12031DC62C83162130AA00AB0183127C
:101968008A01B42283162330AA00AB0183128A01AC
:10197800B4228316A80A0319A90A8A150A1283121F
:10198800031D9F2C0730A300D0308A012F218A0124
:101998000E248A018A2783160430E9000A30ED00F4
:1019A8003230EC000A30EB007830EA0083128A15F6
:1019B8000A122F208A01DE2783162030A800A901E9
:1019C800AA01AB01C30183126400063083164302E7
:1019D8008A150A12831203181B2D83164308053C27
:1019E8008A150A128312031C0E2D8A150A12022563
:1019F8008316BB0083128A150A120E2D0D308A0039
:101A080083164308831282075334593453345434A9
:101A180045344D348A01C52608308316A8070318B3
:101A2800A90AC30A8A150A128312031DE82C831611
:101A3800A801A9011030AA00AB01C30183126400F8
:101A48000430831643028A150A1283120318542D90
:101A580083164308033C8A150A128312031C472D78
:101A68008A150A123D258316BB0083128A150A12AD
:101A7800472D0D308A008316430883128207543499
:101A880045344D3450348A01C52608308316AA07D8
:101A98000318AB0AC30A8A150A128312031D232DE1
:101AA80083162030A800A9013830AA00AB01C30171
:101AB800831264000630831643028A150A128312C1
:101AC8000318902D83164308053C8A150A128312C1
:101AD800031C832D8A150A1277258316BB008312EF
:101AE8008A150A12832D0D308A0083164308831243
:101AF800820748344F34553452344C3459348A01AF
:101B0800C52608308316A8070318A90AC30A8A1528
:101B18000A128312031D5D2DFF3083166C07AA007D
:101B2800FF300318013EAB006B08A800A90183121F
:101B3800831628088312A000831629088312A1009F
:101B480083166A0883128A016E218A150A12031DF8
:101B5800132E831622088312A000831623088312EB
:101B6800A1008A01092120088316A20083122108F6
:101B78008316A3006400803022028A150A12831299
:101B8800031CD12D01308316AA020030031C013E2C
:101B9800AB0283128A150A12D62D8316AA0A0319D4
:101BA800AB0A831283162A088312A00083162B0817
:101BB8008312A10083166C0883128A0172218A1588
:101BC8000A12031DF02DFF3083166C07AA00FF30A0
:101BD8000318013EAB00831283162A088312A00063
:101BE80083162B088312A10083166D0883128A01BD
:101BF8006A218A150A12031D082E013083166D0703
:101C0800AA00AB01AB0D83128A01B4228316A80A7D
:101C18000319A90A8A150A128312031D9C2D83161B
:101C28007A30A800A9011830AA00AB01C3018312B9
:101C380064000D30831643028A150A1283120318B2
:101C4800562E831643080C3C8A150A128312031C6D
:101C5800492E8A150A1236268316BB0083128A1566
:101C68000A12492E0E308A0083164308831282070F
:101C78005434653472346D3469346E3461346C3480
:101C880020344D346F34643465348A01C5260830F5
:101C98008316A8070318A90AC30A8A150A12831209
:101CA800031D1C2E83167830A800A9012030AA0035
:101CB800AB01C301831264000D30831643028A15F9
:101CC8000A1283120318992E831643080C3C8A15AE
:101CD8000A128312031C8C2E8A150A12792683167F
:101CE800BB0083128A150A128C2E0E308A008316C6
:101CF8004308831282075734613469347434693471
:101D08006E3467342E342E342E342E342E342E3442
:101D18008A01C52608308316A8070318A90AC30A2A
:101D28008A150A128312031D5F2E83167A30A800C3
:101D3800A9012830AA00AB01C301831264000E3048
:101D4800831643028A150A1283120318DD2E83169E
:101D580043080D3C8A150A128312031CD02E8A15DB
:101D68000A12BC268316BB0083128A150A12D02ECB
:101D78000E308A0083164308831282075534733461
:101D88006534203447344C345534543449344C3455
:101D9800203431342E3432348A01C5260830831673
:101DA800A8070318A90AC30A8A150A128312031D71
:101DB800A22E0730BA004030B8002030AA00AB018C
:101DC800AE01AF0152308A019B2065308A019B2009
:101DD80061308A019B2064308A019B2079308A0116
:101DE8009B203A308A019B200A308A019B200D30C3
:101DF8008A019B200730BA008030B8002030AA0042
:101E0800AB018A0169205D3C8A150A12031D052F62
:101E18008A0169208316DE005E088312A000633001
:101E28008A016521B20083165E088312A000433040
:101E38008A016521B400320834048A110A16031D88
:101E48000C2983165E088312A00073308A0165216D
:101E5800B20083165E088312A00053308A01652100
:101E6800B400320834048A110A16031D1729831690
:101E78005E088312A00071308A016521B2008316C2
:101E88005E088312A00051308A016521B40032082F
:101E980034048A110A16031D232983165E08831247
:101EA800A00074308A016521B20083165E0883128F
:101EB800A00054308A016521B400320834048A1124
:101EC8000A16031D2F2983165E088312A0006C30A2
:101ED8008A016521B20083165E088312A0004C3087
:101EE8008A016521B400320834048A110A16031DD8
:101EF800522983165E088312A00072308A01652178
:101F0800B20083165E088312A00052308A01652150
:101F1800B400320834048A110A16031D46298316B0
:101F28005E088312A00062308A016521B200831620
:101F38005E088312A00042308A016521B40032088D
:101F480034048A110A16031D3A2983165E0883127F
:101F5800A0006B308A016521B20083165E088312E7
:101F6800A0004B308A016521B400320834048A117C
:101F78000A16031D812983165E088312A0006430A7
:101F88008A016521B20083165E088312A0004430DE
:101F98008A016521B400320834048A110A16031D27
:101FA8008A2983165E088312A00065308A0165219C
:101FB800B20083165E088312A00045308A016521AD
:101FC800B400320834048A110A16031D86298316C0
:101FD8005E088312A00070308A016521B200831662
:101FE8005E088312A00050308A016521B4003208CF
:101FF80034048A110A16031D982983165E08831271
:10200800A00075308A016521B20083165E0883122C
:10201800A00055308A016521B400320834048A11C1
:102028000A16031DAA2983165E088312A0007830B9
:102038008A016521B20083165E088312A000583019
:102048008A016521B400320834048A110A16031D76
:102058005A2983165E088312A00079308A01652107
:10206800B20083165E088312A00059308A016521E8
:10207800B400320834048A110A16031D6E29831627
:102088005E088312A00066308A016521B2008316BB
:102098005E088312A00046308A016521B400320828
:1020A80034048A110A16031DB92983165E0883129F
:1020B800A00068308A016521B20083165E08831289
:1020C800A00048308A016521B400320834048A111E
:1020D8000A16031DCA2983165E088312A0007630EB
:1020E8008A016521B20083165E088312A00056306B
:1020F8008A016521B400320834048A110A16031DC6
:102108001D2A83165E088312A0006D308A0165219E
:10211800B20083165E088312A0004D308A01652143
:10212800B400320834048A110A16031D722B831670
:102138005E088312A0006E308A016521B200831602
:102148005E088312A0004E308A016521B40032086F
:1021580034048A110A16031D292B83165E0883127C
:10216800A0006F308A016521B20083165E088312D1
:10217800A0004F308A016521B400320834048A1166
:102188000A16031D842A83165E088312A000613094
:102198008A016521B20083165E088312A0004130CF
:1021A8008A016521B400320834048A110A16031D15
:1021B8008A2A83165E088312A00067308A01652187
:1021C800B20083165E088312A00047308A01652199
:1021D800B400320834048A110A16031D7D2A8316B6
:1021E8005E088312A00077308A016521B200831649
:1021F8005E088312A00057308A016521B4003208B6
:1022080034048A110A16031D762A8A150A12DD2E4D
:102218008A150A1242228A150A121F238A0180246B
:102228008A150A12DD2E8A150A1242228A150A1206
:102238001F238A150A1259218A150A12DD2E8A15BA
:102248000A1242228A150A121F238A150A12082125
:102258008A150A12DD2E8A150A1242228A150A12D6
:102268001F238A01FA248A150A12DD2E8A150A12FA
:10227800B5228A150A129C228A150A1282208A150A
:102288000A12DD2E8A150A12B5228A150A129C2214
:102298008A150A12B9208A150A12DD2E8A150A1221
:1022A800B5228A014B258A150A12DD2E8A150A12D3
:1022B80042227F088316EB003608EA003708ED0053
:1022C80083128A150A129C228A150A122F208A154F
:1022D8000A12DD2E8A150A1242227F088316ED00A3
:1022E8003608EC003708EB0083128A150A129C2284
:1022F8008A01DE278A150A12DD2E8A013C248A15F6
:102308000A12DD2E83160130E80083128A150A129C
:10231800F6218A150A1228238A01B4228316E801B5
:1023280083128A150A12DD2E8A150A12F6218A15D9
:102338000A1228238A150A129C2283164008BB0019
:1023480083128A01C5268A150A12DD2E8A150A12F9
:1023580042228A150A12282383163708BE008312E0
:102368008A0163278A150A12DD2E8A150A129C2211
:102378008316CF01EF30D000D2013F30D300831253
:102388008A150A1282208A150A12DD2E8A150A1267
:10239800F6218A150A1228238A01782683165108FD
:1023A800EE0083128A150A129C22640083164008E4
:1023B800403C8A110A16831203191A2A64008316EC
:1023C80040083B3C8A110A168312031DF429831620
:1023D8002030BB0083128A01C5268A110A16FA2901
:1023E80083164008BB0083128A01C526083083166D
:1023F800A8070318A90A28088312A0008316290829
:102408008312A100A301EF308A0173218A110A16F1
:10241800031D122A83166E08D10083128A017826BA
:102428008A150A129C228A110A16D9298A150A12B3
:10243800DD2E8A150A12F6218A150A122823831618
:102448002808EE002A08EF0083128A0178268A15E8
:102458000A129C22640083164008403C8A110A161E
:1024680083120319732A6400831640083B3C8A11BF
:102478000A168312031D492A83162030BB008312D3
:102488008A01C5268A110A164F2A83164008BB00FE
:1024980083128A01C52683166E08A800A901083090
:1024A800AA070318AB0A2A088312A00083162B0870
:1024B8008312A100A3013F308A0173218A110A16F1
:1024C800031D6B2A83166F08AA00AB0183128A01C9
:1024D80078268A150A129C228A110A162E2A8A152B
:1024E8000A12DD2E83160230C20083128A110A16E0
:1024F8008E2A83160330C20083128A110A168E2A86
:102508008316C20183128A110A168E2A8316013095
:10251800C20083128A150A12B52283164F08831245
:10252800F600831650088312F500831652088312AA
:10253800F800831653088312F7007508F30076082D
:10254800F4007308A0007408A1007808A3007708B5
:102558008A016F218A110A16031D232B6400831632
:102568004208003C8A110A168312031DD52A8A15CF
:102578000A12B8210730BA001030B8000730BB0083
:102588000830B900A0308A01202074088A01202070
:1025980073088A0120207F088A011E200A308A01D8
:1025A8002E21640083164208013C8A110A16831200
:1025B800031DF72A0730BA001030B8000730BB00F7
:1025C8000830B900A0308A01202074088A01202030
:1025D80073088A0120208A0105208316C00083120F
:1025E8008A150A12A221640083164208023C8A1145
:1025F8000A168312031D0A2B8A150A12B8217308BA
:1026080003178D0003137F088A01202164008316B5
:102618004208033C8A110A168312031D1C2B7308F7
:102628008A0118218316C00083128A150A12A22172
:10263800F30A0319F40A8A110A16031DA52A831638
:10264800C20183128A150A12DD2E8A150A12B522D2
:1026580083165208AA00AB01831283162A08831234
:10266800A00083162B088312A10083165308831237
:102678008A016E218A110A16031D6F2B83164F08D3
:10268800A800A9018312831628088312A0008316C4
:1026980029088312A1008316500883128A016E212B
:1026A8008A110A16031D662B8A01AA228A150A12A4
:1026B800A2218316A80A0319A90A8A110A168312E5
:1026C800031D472B8316AA0A0319AB0A8A110A1697
:1026D8008312031D312B8A150A12DD2E8A150A1260
:1026E800B52283165208AA00AB01831283162A0862
:1026F8008312A00083162B088312A10083165308A7
:1027080083128A016E218A110A16031DBC2B8316B7
:102718004F08A800A9018312831628088312A00075
:10272800831629088312A1008316500883128A0190
:102738006E218A110A16031DB32B8A150A12B821B5
:102748007F088316BE0083128A0163278316A80AAE
:102758000319A90A8A110A168312031D902B8316DE
:10276800AA0A0319AB0A8A110A168312031D7A2BC7
:0827780063008A110A16BC2B54
:02400E00753FFC
:00000001FF
